:10049B00000102030405060708090A0B0C0D0E0FD9
:1004AB00101112131415161718191A1B1C1D1E1FC9
:1004BB00202122232425262728292A2B2C2D2E2FB9
:1004CB00303132333435363738393A3B3C3D3E3FA9
:1004DB00404142434445464748494A4B4C4D4E4F99
:1004EB00505152535455565758595A5B5C5D5E5F89
:1004FB006061626364656667696B6D6F707172735F
:10050B00747576777B7C7D7E7F8081828384858604
:10051B008788898A8B8C8D8E8F90919293949596E8
:10052B009798999A9B9C9D9E9FA0A1A2A3A4A5A6D8
:10053B00A7A8A9AAABACADAEAFB0B1B2B3B4B5B6C8
:10054B00B7B8B9BABBE0E1E3E4F0F1F21201000194
:10055B000000000800055BC31248000000010902FF
:10056B002E0001010080C8090400000400000000F7
:10057B00070581024000FF070502024000FF070547
:0C058B0085024000FF070506024000FF4B
:10027800750900750A0085260BE527249F7003027F
:10028800038414700302038714700302039924F291
:10029800700302033314603E24FE700302037224C9
:1002A800FD60582410600302039EE42526FFE43411
:1002B8007EFE120D4F8F087D087F2B7E7E120D5E0D
:1002C800AD087F297E7E120D5E3011057D07020381
:1002D8006B7D0302036B7D087F2B7E7E120D5EAB68
:1002E80009AA0AA90B1209D0FD7F297E7E120D5E8C
:1002F8003011047D0780027D038068AB09AA0AA932
:100308000BE52A120A167D087F2B7E7E120D5EAB46
:1003180009AA0AA90B1209D0FD7F297E7E120D5E5B
:100328003011047D0780027D038038852A457B01D2
:100338007A007982AF4512004C7D087F2B7E7E12B1
:100348000D5E900082E0FD7F297E7E120D5E90009A
:1003580083E0FD7F297E7E120D5E3011047D0780CB
:10036800027D037F2B7E7E020D5E852A458525440E
:10037800852643AB25AD26AF2A020071D206227B23
:10038800007A00794812111E7B007A007948020F22
:0703980004AF2A1211B92283
:1011890075A0BE12107A1210881210881210887574
:08119900A0FE1210880210886C
:10087600E4F520C200F535F534F53F7D01FF7E7EB7
:10088600120D5E7F007E7E120D4FEF20E0F57DC4D7
:100896007F007E7E120D5EE4FD7F077E7E120D5E7A
:1008A6007D057F017E7E120D5E7D107F0F7E7E129E
:1008B6000D5E7D0F7F0B7E7E120D5E7D0F7F0D7EA2
:1008C6007E120D5E7D507F097E7E120D5E7DD67F87
:1008D600077E7E120D5EE4FD7F167E7E120D5E7D26
:1008E600407F1F7E7E120D5E7D807F047E7E120D10
:1008F6005EE4FD7F207E7E120D5E7D087F237E7E78
:10090600120D5E7D017F277E7E120D5E7D027F05C4
:0E0916007E7E120D5E7DCC7F007E7E020D5E29
:100CE7007F087E7E120D4F8F2DE52D30E62FE4FD18
:100CF7007F057E7E120D5E7D807F047E7E120D5EF7
:100D0700E4FD7F207E7E120D5E7D087F237E7E12AE
:100D17000D5E7D017F277E7E120D5E8018E52D54C6
:100D270030600D7DC07F097E7E120D5E7D038010D1
:100D3700E52D30E7127D507F097E7E120D5E7D0224
:080D47007F057E7E120D5E2285
:100F4700E537540324FE7037E53AB4070050309074
:100F57000F5DF8282873020F72020F75020F7802CF
:100F67000F7B020F7E020F81020F84C20822C20983
:100F770022C20A22C20B22C20C22C20D22C20E2298
:1010B300D200853A36E536B401057533128008E56A
:1010C30036B4020375332EE533D3953D4003853D96
:1010D30033E4F524E524C39533500C12114C052455
:0810E300E524C3940840ED224E
:10114C00E536B40107E524900557800AE536B4026C
:10115C0008E52490056993F509AD097F217E7E028F
:02116C000D5E16
:10092400E537540314600A14600E240260030209BC
:10093400C78000E4FD0209C0E53AB40700400302A1
:1009440009C790094DF828287302096202096E024A
:10095400097C02098A0209980209A60209B4E52160
:1009640060047D018002E4FD8052E521640160049D
:100974007D018002E4FD8044E521640260047D0180
:100984008002E4FD8036E521640360047D01800279
:10099400E4FD8028E521640460047D018002E4FD17
:1009A400801AE521640560047D018002E4FD800C69
:1009B400E521640660047D018002E4FD7F217E7EE2
:0C09C400120D5EE4FD7F217E7E020D5EC0
:10070C00853935E5396077E4F522F5217D087F2BB5
:10071C007E7E120D5E7D117F287E7E120D5E7D0821
:10072C007F2F7E7E120D5E7D127F2C7E7E120D5EE3
:10073C007D017F2F7E7E120D5E7D087F3B7E7E12BB
:10074C000D5E7D157F307E7E120D5E7D157F387EB1
:10075C007E120D5E7D087F3F7E7E120D5E7D167FC4
:10076C00347E7E120D5E7D017F377E7E120D5E7DA6
:10077C00167F3C7E7E120D5E7D017F3F8031E4FD55
:10078C007F287E7E120D5EE4FD7F2C7E7E120D5E38
:10079C00E4FD7F307E7E120D5EE4FD7F347E7E12A2
:1007AC000D5EE4FD7F387E7E120D5EE4FD7F3C7EA7
:0507BC007E120D5E221B
:100F8700E537540324FE7037E53AB4070050309034
:100F97000F9DF8282873020FB2020FB5020FB8028F
:100FA7000FBB020FBE020FC1020FC4D20822D20923
:100FB70022D20A22D20B22D20C22D20D22D20E2208
:1010EB00D2027D087F2B7E7E120D5E7A0079827C88
:1010FB00007D827B407F297E7E120D92752E0075BE
:10110B002F403011047D0780027D037F2B7E7E12E2
:03111B000D5E2244
:100C7A00D204D2057D087F337E7E120D5E7A00791A
:100C8A0082E5182482FDE5173400FC7B407F317E23
:100C9A007E120D927D087F3B7E7E120D5E74C22508
:100CAA0018F58274003517AD82FC7B407F397E7E51
:100CBA00120D927540007541807D157F307E7E123F
:100CCA000D5E7D157F387E7E120D5E7D037F337E3D
:0D0CDA007E120D5E7D077F3B7E7E020D5E6B
:10111E008B0C8A0D890EE4F50FE4250FFFE4347E67
:10112E00FE120D4FAB0CAA0DA90E850F8275830012
:0E113E00EF120A28050FE50FC3944040DC2293
:100F04008B0C8A0D890E7D087F2B7E7E120D5EE48C
:100F1400F50FAB0CAA0DA90E850F8275830012097B
:100F2400E9FD7F297E7E120D5E050FE50FC3943F18
:100F340040E03011047D0780027D037F2B7E7E120A
:030F44000D5E221D
:1007C1007F267E7E120D4F8F28E52820E603020842
:1007D1005EE4F5307F257E7E120D4F74372530F8AB
:1007E100A6070530E530C3940840E97D087F277EE0
:1007F1007E120D5E7D087F237E7E120D5EE53754ED
:1008010060704EE538602624FD604324FE602314A9
:10081100601624FE600C14603024087034120F47F7
:10082100802FAD357F21801A1210B3802412092444
:10083100801F7D407F207E7E120D5EE5394480FD64
:100841007F047E7E120D5E800812070C8003120F5A
:10085100877D057F237E7E120D5EC2102230000B44
:10086100C2007D087F237E7E120D5E7D017F277E83
:050871007E120D5E2265
:100B90007F2E7E7E120D4F8F28E52820E653E52814
:100BA00020E74ED2017F2D7E7E120D4F8F2C7F2DA0
:100BB0007E7E120D4F8F277F2D7E7E120D4F8F2A46
:100BC0007F2D7E7E120D4F8F257F2D7E7E120D4F45
:100BD0008F267F2D7E7E120D4F8F2BE52CB4AA0F12
:100BE0002527252A25252526F52B6003120278C204
:100BF000012002127D087F2F7E7E120D5E7D017F17
:070C00002F7E7E120D5E2223
:100EBD007F367E7E120D4F8F28E52820E70630E421
:100ECD000330E50F7D087F377E7E120D5E7D017F3D
:100EDD0037801E7A0079007C007D007B407F357E57
:100EED007E120D6D7D087F377E7E120D5EE4FD7FD7
:070EFD00347E7E120D5E221F
:100AFD007F3E7E7E120D4F8F28E52820E70630E4DD
:100B0D000320E5127D087F3F7E7E120D5E7D017F05
:100B1D003F7E7E020D5E7A0079407C007D407B3DFC
:100B2D007F3D7E7E120D6D7D087F3F7E7E120D5EB8
:100B3D007D017F3F7E7E120D5E7D167F347E7E129F
:100B4D000D5E7D017F377E7E120D5ED21890000006
:100B5D00E0139206E0FF74C6251CF5827401351B67
:100B6D00F583EFF074C7251CF5827401351BF583F1
:100B7D00E516F074C8251CF5827401351BF583E567
:030B8D001AF02239
:100DB7007F227E7E120D4F8F29E52930E64F30E5E1
:100DC7004C7D087F237E7E120D5E300037E524249C
:100DD70008F508E524C39508500EE524C39533505C
:100DE7000712114C052480EBE53314B52403E4F511
:100DF700243010047D0580027D017F237E7E120D45
:0E0E07005EB210227D017F277E7E120D5E22DC
:100A68007F2A7E7E120D4F8F29E52920E603020A90
:100A7800FC20E503020AFCB2117D087F2B7E7E1262
:100A88000D5E30025DE52F2440FFE4352EFEC3EFF6
:100A9800947CEE940250047F408006C3747C952FAA
:100AA800FF8F087482252FF5827400352EAD82FCE5
:100AB800AB087F297E7E120D92E508252FF52FE4DD
:100AC800352EF52EE52FB47C0CE52EB40207E4F59F
:100AD8002EF52FC2023011047D0780027D037F2B83
:100AE800800D7D087F2F7E7E120D5E7D017F2F7E1B
:050AF8007E120D5E22DC
:100597007F327E7E120D4F8F29E52920E603020662
:1005A7004420E5030206447D087F337E7E120D5EFC
:1005B700300470E4FD7F307E7E120D5EE5412440FD
:1005C700FFE43540FEC3EF9460EE940150047F4092
:1005D7008006C374609541FF8F0874822518F582E1
:1005E70074003517F583E5822541F582E5833540AB
:1005F700AD82FCAB087F317E7E120D92E508254166
:10060700F541E43540F5407D037F337E7E120D5E74
:10061700E54164607004E54064017032F540F541DE
:10062700C20422C205E4FD7F307E7E120D5E7D0886
:100637007F377E7E120D5E7D017F37800CE5292096
:0F064700E60C30E5097D137F337E7E120D5E22B7
:100656007F3A7E7E120D4F8F29E52920E60302069A
:10066600FA20E5030206FA7D087F3B7E7E120D5EC8
:100676003004707D157F307E7E120D5EE54124408C
:10068600FFE43540FEC3EF9460EE940150047F40D2
:100696008006C374609541FF8F0874822518F58221
:1006A60074003517F583E5822541F582E5833540EB
:1006B600AD82FCAB087F397E7E120D92E50825419E
:1006C600F541E43540F5407D077F3B7E7E120D5EA9
:1006D600E54164607004E54064017029F540F54128
:1006E600C20422C2057D087F3F7E7E120D5E7D011B
:1006F6007F3F800CE52920E60C30E5097D177F3B1E
:060706007E7E120D5E2252
:1011A100300014C2007D087F237E7E120D5E7D011A
:0811B1007F277E7E120D5E22F5
:0100060022D7
:0100070022D6
:0100080022D5
:0300030002039F56
:10039F00C0E0C0F0C083C082C085C084C0867586AF
:1003AF0000C0D075D000C000C001C002C003C0049F
:1003BF00C005C006C0077F067E7E120D4F8F2DE54C
:1003CF002D30E6337F0C7E7E120D4F8F2DE52D30B5
:1003DF00E0061207C102047AE52D30E106120B90F8
:1003EF0002047AE52D30E205120EBD807EE52D3038
:1003FF00E379120AFD8074E52D30E2317F0A7E7EAB
:10040F00120D4F8F2DE52D30E005120DB7805CE5F5
:10041F002D30E105120A688052E52D30E2051205F4
:10042F00978048E52D30E343120656803EE52D3088
:10043F00E105120CE78034E52D30E42F7F0E7E7E30
:10044F00120D4F8F2DE52D30E4051211A1801CE503
:10045F002D30E5051200068012E52D30E60512005D
:10046F00078008E52D30E703120008D007D006D02B
:10047F0005D004D003D002D001D000D0D0D086D088
:0C048F0084D085D082D083D0F0D0E03241
:100E6C00E4F512900001E0FFE512C39F5042E51239
:100E7C0075F003A42402F582E43400F583E0F51345
:100E8C00E51275F003A42403F582E43400F583E045
:100E9C00F515E51275F003A42404F582E43400F58D
:100EAC0083E0F514FBAD15AF13120088051280B367
:010EBC002213
:1011B900EF146011047010C2A9E4F51AF516FBFDCD
:0811C9007F7F020071D2A92210
:10002600540FB40A0040022407243022F546C412B5
:100036000026F5993099FDC299E546120026F599F4
:100046003099FDC29922C2AF8C838D828F8075A0B4
:10005600EF75A0EE7580FF7590FF75A0E200E58054
:10006600F0E590A3F075A0FED2AF22C2AF8F8075E7
:10007600A0EF75A0EE8B808D9075A0E875A0FED2DE
:10008600AF228F8075A0EF75A0EE008B808D9075E6
:10009600A0E80075A0FE0022898075A0EF75A0EE8D
:1000A6007580FF75A0E200E580F0B98301FCE5905C
:1000B600F0B98301FD75A0FE22C083C0828E838FB6
:1000C600824386107590FF790012009E09B930F9B7
:1000D6005386EFD082D08322C083C0828E838F82E4
:1000E6004386107590FF790712009EE92408F9B936
:1000F60037F65386EFD082D08322C083C0828E83A8
:100106008F824386107590FF798012009E09B9840C
:10011600F9798412009E09B99CF95386EF7B85BB59
:100126009D02214AEC30E0148B8075A0EF75A0EE9D
:1001360075800075900075A0E875A0FE03FC740438
:090146002BFB2125D082D083227D
:0D11D10043C28043C401538EF8438E0222B6
:101041001211D17FFF12000E12116ED2AFD2A8D2AF
:10105100AC121189120876E4F542F523C2A9D2B97E
:101061001210055320BFE52030E6FB30E7F8120CE3
:091071007A5320BF53207F80ED6B
:10107A00751D4BD51DFD22751D04D51DFD22751F3D
:10108A001412107AD51FFA22751D2D751EFFD51E52
:10109A00FDD51DF722751F28121092D51FFA227549
:0910AA001FA012107AD51FFA22D2
:10000E00759850D29C4389208F8D8F8BD28EC2993A
:04001E004387802272
:100FC700EF7804A2E713D8FB540FFEC36480948A1A
:100FD700EE50062430F59980042437F5993099FDB1
:100FE700C299EF540FFEC36480948AEE50062430F2
:0E0FF700F59980042437F5993099FDC29922AE
:10116E00E4FFFE74822FF58274003EF583EFF00FDC
:0B117E00BF00010EBE02ECBFC0E92262
:100C0700E5996461702BFCFD75997C3099FDC2995B
:100C1700AF05120FC774822DF58274003CF583E08F
:100C2700FF120FC70DBD00010CBC02DCBDC0D9808F
:100C37002FE59964637029FCFD75997C3099FDC295
:100C470099AF05120FC774002DF58274003CF58328
:100C5700E0FF120FC70DBD00010CED64824C70D987
:100C670075990D3099FDC29975990A3099FDC29908
:030C7700C29822FE
:03002300020E15B5
:100E1500C0E0C083C082C085C084C086758600C01E
:100E2500D075D000C000C004C005C006C00730980A
:100E35001D120C078599993099FDC29975990D3048
:100E450099FDC29975990A3099FDC299C298D00742
:100E5500D006D005D004D000D0D0D086D084D0859F
:070E6500D082D083D0E032FF
:100D4F00C083C0828E838F82E0FFD082D08322C087
:100D5F0083C0828E838F82EDF0D082D08322C083B6
:100D6F00C082BB0001227586048E838F8205868C1C
:100D7F00858D840586E00586F0A3DBF70586D08296
:100D8F00D08322C083C082BB0001227586048E836C
:100D9F008F8205868C858D84E0A30586F00586DB22
:080DAF00F70586D082D08322F3
:10100500E4F51AF516F519E5165401FF7E007C0185
:101015007D60120A4A8E1B8F1CE5162401FF7E0097
:10102500EF5401FF120A4A8E178F185389F143892D
:0C10350001C28C758CF9758A8DD28C225A
:03000B0002014FA0
:10014F00C0E0C0F0C083C082C085C084C086758601
:10015F0000C0D075D000C000C001C002C003C004F1
:10016F00C005C006C007C2AFC28C758CF9758A8DE9
:10017F00D28CE51A75F038A485F010F511E4FBFD6B
:10018F007F801200887482251CF5827400351BF560
:10019F0083E5822511F582E5833510AF82FE1201CA
:1001AF0000E51C2511FFE51B3510FE74892FF58224
:1001BF0074003EF583E030E5137462251CF58274FC
:1001CF0001351BAF82FE1200BF751901E519701BB7
:1001DF007462251CF5827401351BF58375F00CE5EF
:1001EF001A120A5CAF82AE831200DE7E00E51C2578
:1001FF001AFFEE351BFE74C22FF58274013EF58394
:10020F00E516F0051AE51AC39404403AE52330E0E9
:10021F0006120E6C5323FE751A007519000516E5AC
:10022F00165401FF7E007C017D60120A4A8E1B8FDF
:10023F001CE5162401FF7E00EF5401FF120A4A8EBF
:10024F00178F18432080D2AFD007D006D005D00427
:10025F00D003D002D001D000D0D0D086D084D085AA
:09026F00D082D083D0F0D0E0323F
:030000000211DE0C
:0C11DE00787FE4F6D8FD7581870210418F
:1009D000BB010689828A83E0225002E722BBFE0225
:0909E000E32289828A83E4932258
:1009E900BB010CE58229F582E5833AF583E02250C3
:1009F90006E92582F8E622BBFE06E92582F8E2220D
:0D0A0900E58229F582E5833AF583E4932226
:100A1600BB010689828A83F0225002F722BBFE01BF
:020A2600F322B9
:100A2800F8BB010DE58229F582E5833AF583E8F004
:100A3800225006E92582C8F622BBFE05E92582C8B0
:020A4800F22298
:100A4A00EF8DF0A4A8F0CF8CF0A428CE8DF0A42EC0
:020A5A00FE227A
:0C0A5C00A42582F582E5F03583F58322A5
:00000001FF
